:1000000000308A00642A00000A108A100A11820750
:1000100028340C34013406340A108A100A1182077D
:1000200047345034533452344C3430343134423405
:1000300020340A3400340A108A100A118207283446
:100040006334293420344B3461346B346C34693478
:100050006B342034323430343034383400340A10C5
:100060008A100A1182070C340034CE308400000854
:10007000031949280130F800F701F70B3D28F80B68
:100080003C284A30F700F70B432800000000800BA3
:100090003A28003406080F398316D500540EF700AD
:1000A000F030F7057708F0395504831286000615FD
:1000B000831606112130F700F70B5C288312061116
:1000C00083160611831200348316D208031D6C2890
:1000D000831286106E288316831286148316861068
:1000E000D30E5308D40083124A208316D30E53082C
:1000F000D40083124A204230F700F70B7D2800001D
:10010000003414308316CE00831235200F3083164E
:1001100086058312861083168610831206118316B5
:100120000611CC014C08023C031CA2280230CE0070
:100130008312352003308316D40083124A2083169D
:10014000CC0A92280D30F700F70BA4280230D40017
:1001500083124A200D30F700F70BAC288316CC0130
:100160004C08023C031CC6284C088312042083164A
:10017000CD00D2014D08D3008312642002308316D3
:10018000CE00831235208316CC0AB02883128A1140
:100190000A12C72A013083164F02FC3E0318E328D7
:1001A000043E8312EF288316D001E32840308316E3
:1001B000D000E32814308316D000E328543083168F
:1001C000D000E328831601304E02D0075008803853
:1001D000D100D2015108D3008312642000340A10E8
:1001E0008A100A118207D328D628DA28DE28831637
:1001F0004D080C3A831203190729063A03191329EB
:10020000073A03191B29053A0319222929298316BC
:10021000D2010130D3008312642002308316CE0055
:1002200083123520372901308316CE000230CF00EB
:100230008312CA20372901308316CE00CF008312E3
:10024000CA2037298316D2011030D30083126420CC
:10025000372983164D081F3C031C30290730CD0574
:100260000130D2004D08D3008312642037290034B6
:100270000830F70020172008831687008312071F15
:10028000432983163E298316CF01F7175729F71301
:10029000572903108312071B03148316CF0C7717FB
:1002A00057297713F70B49294F08F80062293F3087
:1002B000F71B1130F800F80B5B29F71B4729771B58
:1002C000512949298312003483164D08CF004F0865
:1002D0008400800803196E29CF0A67294E0884001C
:1002E000800803197E294E0884000008D1004F08B9
:1002F000840051088000CF0ACE0A6E294F0884007E
:1003000080014D08F80083120034A01320088316E2
:100310008700831287130830F800000000000000F7
:10032000F817A329F8138316D50C8312031887171F
:10033000031C87137817A3297813F80B932900005F
:100340000000000087171C308400840BA5290000E2
:100350000000F81B9229781B9C2900348316500852
:10036000F8014F020318B7294F08F700C329F70116
:100370000830D100CF0DF70D500877020318F700B1
:10038000F80DD10BBA2983120034780883164D0872
:10039000CF006430D0008312AE2177088316CD00E1
:1003A00078083030031DDB29CE1CE429CE19E4295E
:1003B0004E1A2030DE29CE114E124E14F80778085E
:1003C000D5008312852183164D08CF000A30D00056
:1003D0008312AE2177088316CD0078083030031DD4
:1003E000F729CE19FD294E1CFD294E1A2030F80799
:1003F0007808D5008312852183163030CD074D084B
:10040000D500831285218A110A12822C04088316D2
:10041000D4004E0EF038D000D007E23ED100323E7C
:10042000D3004E080F39D107D107D307E93ED200D8
:10043000D207D2074D0E0F39D207D307D20DD30DF5
:10044000D309D30D4D080F39D307D00D0730CF0096
:100450000A30D307D203031C292AD207D103031C75
:100460002D2AD107D003031C312AD007CF03031C48
:10047000352ACF3084000730540554138407D33015
:100480000402031954170008F700031D4F2A541BD8
:100490004F2A541A5D2AD4194F2A2030522AD415D3
:1004A00054123030F707CE010408CD007708D5008C
:1004B0008312852183164D088400840A541F3F2A25
:1004C00083128A110A12922CA701D730A600163087
:1004D0008316D700D901D801831284011F30830508
:1004E0008316051083120514A013200883168700B5
:1004F0008312871783161F149F141F159F1107302F
:100500009C00FF308312A000A1010130A200A301D2
:10051000A401A50183161F109F141F159F151F13FB
:1005200083121F179F1783169F1783121F1494128D
:10053000A012200883168700831220162008831635
:1005400087008312A01120088316870000308312D1
:100550009400831694000108C7390838810083127B
:1005600090010030F80092000030831692000730AE
:100570009C0005080330F700F70BBC2A1C08831207
:100580000D13FE3083169D000515831281286430FB
:100590008316CE008312352005308316CE0001303D
:1005A000CF008312CA20E80168080C200038031924
:1005B000DF2AE80A8316CD008312F720D42AE80147
:1005C00068081B2000380319EB2AE80A8316CD00BF
:1005D0008312F720E02A0230E80096308316CE001E
:1005E00083123520E80BED2AE80168082F20003837
:1005F0000319002BE80A8316CD008312F720F52A91
:100600000830F8001F08C73978049F00BB01CF01EC
:10061000E3018316B301C701831238217808243C13
:100620000319142B83160C2B1F151F19152B83165A
:100630001E088312E5001E08E6002430A8000130E1
:10064000E4006408123C031C302B2830640784004B
:10065000E90038216908840078088000E40A212B29
:10066000E4016408123C031C402B3C306407840006
:10067000E90038216908840078088000E40A312BF9
:10068000E4016408123C031C502B503064078400C2
:10069000E90038216908840078088000E40A412BC9
:1006A000E4016408123C031C772B38217808E7002A
:1006B00067082A3C031D702BA0306407840080016A
:1006C00067088316B4008312382178088316B500B2
:1006D0008312382178088316B600B701AA2B83123B
:1006E000A0306407840067088000E40A512BE4010D
:1006F0006408123C031CA92B38217808E70067081E
:100700002A3C031DA22BB4306407840067088000D4
:1007100001306407B43E8400EA0038216A0884008E
:100720007808800002306407B43E8400EA00382173
:100730006A0884007808800003306407B43E8400AF
:100740008001A92BB4306407840067088000E40AA4
:10075000782B83168312E80168082F2000380319CC
:10076000B72BE80A8316CD008312F720AC2B201498
:1007700020088316870083120718EC2B013083169C
:10078000CE00CF008312CA2028308400003000043D
:100790000319D52B0408E80000088316CD00831246
:1007A000F72068088400840AC62B0A308316CD001F
:1007B0008312F7203C308400003000040319EB2B37
:1007C0000408E80000088316CD008312F7206808AB
:1007D0008400840ADC2B192C01308316CE00CF0054
:1007E0008312CA2050308400003000040319032C07
:1007F0000408E80000088316CD008312F72068087B
:100800008400840AF42B0A308316CD008312F7206B
:10081000A0308400003000040319192C0408E800FB
:1008200000088316CD008312F72068088400840A2C
:100830000A2C3C308316CD005030CE008312642148
:100840007808E80028308316CD00831278088316D4
:10085000CE00831264217808E9008400003000048F
:1008600003193D2C0408EA0000088316D500831202
:1008700085216A088400840A2E2C0D308316D50049
:10088000831285210A308316D50083128521A0307A
:100890008316CD00B430CE00831264217808E800BE
:1008A0008400003000040319602C0408E9000008EB
:1008B0008316D5008312852169088400840A512C8F
:1008C0000D308316D500831285210A308316D5009A
:1008D000831285218316051600308312051A013014
:1008E000E80020308316D500831285212F3083162F
:1008F000D5008312852168088316CD001B30CE00F9
:100900008312C5292F308316D5008312852110301C
:10091000840066088316CE00831265088316CD0016
:100920008312062A0A308316D500831285210D30E2
:0C0930008316D50083128521062B63007E
:02400E00393F38
:00000001FF
